:10000000412883169B0083161C141A089B0A3D285E
:1000100083169A001C1555309D00AA309D009C1433
:100020009C1810281C119B0A3D288001840AFF3E61
:10003000031D15283D28A401A300FF30A307031CBE
:10004000A407031C3D280330A200DF3029201D280F
:10005000A201E83EA100A209FC30031C3228A1073E
:1000600003182F28A1070000A20F2F2821183828D5
:10007000A11C3C2800003C280800831383120313B2
:100080000800FF2383169000831207309900850132
:1000900087010830831685008701203084004030B6
:1000A0008312152064301B207A2085160130A400AD
:1000B00090301C200130AA0085195F28AB14013054
:1000C000A200F4302920AA0A031D5C288512AB1C6B
:1000D00079280130AA000A302A0203187828203033
:1000E00085060130A400F4301C20AA0A031D6B28E9
:1000F000AE20C828051205108510051107108710BD
:100100000711871107128712AB188728851208007C
:100110008310851983148318AB15831CAB11AA01B6
:1001200003018519013EAB19013C03190130031D80
:100130000301A50032302A02013003180301A5058E
:100140000319A428AA0A902832302A02031DA928DC
:100150002B140330A200E830292008000130A7004A
:100160002C30A600A608031DB828A7080319C72825
:10017000A603260A0319A7038519C2280130A70080
:100180002C30A6000130A200F4302920B22808004B
:10019000AB18CB288512851DCE28CB28AA010130AB
:1001A00085190301A50034302A0201300318030128
:1001B000A5050319DD28AA0ACF2834302A0203181E
:1001C000E228C82885160230A2005830292088204D
:1001D0000301AB1D013E03192813031D28178820B6
:1001E0002B15AB1D2B1188202916AB1D2912882039
:1001F000A915AB1DA91188202915AB1D291188202F
:10020000A914AB1DA91088202914AB1D2910882022
:10021000A816AB1DA81288202816AB1D281288200E
:10022000A815AB1DA81188202815AB1D2811882002
:10023000A814AB1DA81088202814AB1D28102B1C57
:1002400023292B10C828AB1C262975290030012032
:10025000A00029082002031D7429A808031D3329C2
:1002600010308506732901302802031D3A29013018
:100270008506732902302802031D412902308506B4
:10028000732903302802031D482904308506732989
:1002900004302802031D4F290130870673290530D9
:1002A0002802031D562902308706732906302802CA
:1002B000031D5D2904308706732907302802031DBA
:1002C000642908308706732908302802031D6B292A
:1002D00010308706732909302802031D7229203047
:1002E00087067329C828AE20C82883169B0183126D
:1002F00029080820AB100130AA0015302A02031883
:1003000088292030850696301B20AA0A031D7D29E6
:06031000AE20C8288A2976
:02400E00043E6E
:024200000000BC
:00000001FF
